:020000040000FA
:100000000030650005159901482090309D001A20A8
:1000100018089D001A207F309D001A203B20803058
:100020009D001A2018089D001A207F309D001A207C
:100030003B200428051118309F009F0B1D28083015
:100040009B009D0C03182728000005112A28051580
:100050000000000017309F009F0B2C289B0B2128CD
:100060000000000000000000000005151A309F008D
:100070009F0B382808000D309C00FF309B00FF309C
:100080009A009A0B41289B0B3F289C0B3D280800A7
:0E009000013098070310980D031898060034ED
:02400E00FB3F76
:00000001FF
